:03000000020006F5
:10005F00750800750980750A00750BC0750EC0759F
:0E006F000FC17510D07511D9751200751340B0
:03009B000200035D
:030003000203D520
:10009E00D2B4901C007410F0C2B4D2B4901E00748E
:1000AE00A0F0C2B4D2B4900A007443F0C2B4D2B479
:1000BE00900C007423F0C2B4D2B49008007421F0F6
:1000CE00C2B4D2B49004007413F0C2B4D2B490028D
:1000DE00007430F0C2B422AE82AF83C2B48E828F6F
:1000EE0083E517F022AE82AF83C2B48E828F83E097
:1000FE00F58222AF8253070FBF0A0050068F067497
:10010E00302EFF8F8222AF82BF30004008BF3A00F0
:10011E00500353070F8F8222AE82AF83D2B48E82EA
:10012E008F83E0FEC2B4E5145206EEC4540FF5827E
:10013E00A910C006C001120101E582D001F7A91075
:10014E008782121044D006A9108E82C001120101BE
:10015E00E582D001F7A910878202104475141F9012
:10016E000A0012012675822F12104475143F900852
:10017E000012012675822F1210447514FF900C0088
:10018E0012012675822012104475143F900400123D
:10019E00012675823A12104475147F9002001201E6
:1001AE002675823A12104475147F900000020126C3
:1001BE00850A82850B83D2B4E0FFC2B48F177518FF
:1001CE000090000512133D7517FF7518001213F9F4
:1001DE00AE82751736751801900000C0061204F82D
:1001EE00758201120522751796751800900000127F
:1001FE0004F890146775F0801210B7D006EE9014C4
:10020E004693F5820210447517327518009000005F
:10021E001204F890147375F0801210B7900000124B
:10022E0000F3121044751764751800900000120444
:10023E00F890147B75F0801210B790FFFF1200F348
:10024E000210447F10E50EF876007590F0E590549C
:10025E00F0FEC007C006120486AC82AD83C005C096
:10026E000412048E858215858316120496AB827550
:10027E00172C75180190005AC0031204F8758201EC
:10028E0012052212016A1201BE120215D003D00409
:10029E00D0058515178516188C828D83C003120420
:1002AE00F8D0038B82120522D006D007BEF0028052
:1002BE009975900FE590540FFDA90F4EF77E00BD76
:1002CE000F02801FEE24C3401A75900FAD90900060
:1002DE0014C007C006C00512040DD005D006D00705
:1002EE000E80DC7D00ED90143593FCA90F8703EC96
:1002FE00B503028D070DBD100040EABE3C0040085C
:10030E00BF0E05E50EF876018F8222120251AF82E2
:10031E00BF100122EF90144693FEBE460050188E79
:10032E0082C007121044D007EF90145793FFD2B437
:10033E00908000EFF0C2B4227F0078CC860508864C
:10034E0006758203C007C006C0051205227582021B
:10035E0012053690001412040DE4F517F5189000EE
:10036E00001204F8E4F517F5189007FF12050D12A8
:10037E000CDAE4F517F5189000001204F8901481C9
:10038E0075F0801210B7D005D0068D828E8375174A
:10039E000F751800121314AD82D007A90EE7702145
:1003AE00C3EF9D400E75820AC005121044D0057F22
:1003BE0000800BC007C005120319D005D0070F80AF
:1003CE00DAE50EF876002290FA0012040D90FA008B
:1003DE0012040D758E02C2B5D2B4E50EF876001277
:1003EE00067112009E121222751721900000120043
:0F03FE00E575173F90FFFF1200E512034680FBE5
:101435007DEEEDEBDEDDDBBEBDBBE7D7B7777B7EB3
:10144500003031323334353637383941424344453B
:1014550046003F065B4F666D7D077F6F777C395E83
:1014650079714144432056616C75653A2000537487
:101475006172743A2000456E643A200046726565D3
:0914850020547970653A200A0038
:10007D007521007522407523C27524C47525C6757A
:0E008D0026C77527C87528CA7529CC752ACED6
:10040D00AE82AF837C007D00C3EC9EED64808FF0E7
:10041D0063F08095F050147A507B001ABAFF011BDF
:10042D00EA4B70F70CBC00E00D80DD22AF82C2B547
:10043D00D2B4852182852283EFF0C2B422AF82D25D
:10044D00B5D2B4852182852283EFF0C2B422AF826A
:10045D00852182852283EFF022AF82C2B5D2B48589
:10046D002182852283EFF0C2B4D2B5D2B485218228
:10047D00852283E517F0C2B422A9238782098783D9
:10048D0022A924878209878322A925878222AE8209
:10049D00AF83E523F8A60608A60722AE82AF83E553
:1004AD0024F8A60608A60722AE82AF838F05C2B533
:1004BD00D2B4852182852283EDF0C2B4C2B5D2B407
:1004CD00852182852283EEF0C2B4AF18AE17D2B566
:1004DD00D2B4852182852283EFF0C2B4D2B5D2B4D5
:1004ED00852182852283EEF0C2B422AE82AF83E5F0
:1004FD0023F8A60608A607E524F8A61708A61822CD
:10050D00AE82AF83E527F8A60608A607E528F8A66C
:10051D001708A61822E582FF24F7500122A925EF1E
:10052D00600280027F01A70722AF82E526F8A607A9
:10053D00EF24FC405EEF2F900548738006801880F5
:10054D002A803C7F48E529F876F0087600E52AF800
:10055D007640087601804E7F28E529F876400876AA
:10056D0001E52AF876F0087600803A7F88E529F8CB
:10057D0076F0087600E52AF8764008760180267F29
:10058D00E8E529F87640087601E52AF876F0087650
:10059D000080127F48E529F876F0087600E52AF804
:1005AD007640087601C2B5D2B48521828522837446
:1005BD0036F0C2B4D2B5D2B4852182852283EFF054
:1005CD00C2B422AE82AF83C2B5D2B4852182852258
:1005DD0083742AF0C2B48F05D2B5D2B48521828539
:1005ED002283EDF0C2B4D2B5D2B4852182852283A7
:1005FD00EEF0C2B4AF1AD2B5D2B485218285228372
:10060D00EFF0C2B4AF19D2B5D2B485218285228361
:10061D00EFF0C2B4C2B5D2B4852182852283742B8A
:10062D00F0C2B4AF18D2B5D2B4852182852283EF42
:10063D00F0C2B4AF17D2B5D2B4852182852283EF33
:10064D00F0C2B4AF1CD2B5D2B4852182852283EF1E
:10065D00F0C2B4AF1BD2B5D2B4852182852283EF0F
:10066D00F0C2B422E529F876F0087600E52AF8768E
:10067D0040087601C2B5D2B4852182852283E4F08B
:10068D00C2B4D2B5D2B4852182852283E4F0C2B43E
:10069D00D2B5D2B4852182852283E4F0C2B4D2B51D
:1006AD00D2B4852182852283E4F0C2B49000C812B1
:1006BD00040DC2B5D2B48521828522837401F0C2A6
:1006CD00B490003212040DC2B5D2B48521828522B8
:1006DD00837428F0C2B490000A12040DC2B5D2B4CE
:1006ED0085218285228374C0F0C2B4D2B5D2B4857F
:1006FD0021828522837423F0C2B4C2B5D2B4852180
:10070D008285228374C1F0C2B4D2B5D2B485218260
:10071D008522837411F0C2B4C2B5D2B4852182850D
:10072D00228374C5F0C2B4D2B5D2B485218285229C
:10073D0083743DF0C2B4D2B5D2B4852182852283B3
:10074D007430F0C2B4C2B5D2B485218285228374CF
:10075D00C7F0C2B4D2B5D2B485218285228374AAE2
:10076D00F0C2B4C2B5D2B48521828522837436F02D
:10077D00C2B4D2B5D2B48521828522837488F0C2E9
:10078D00B4C2B5D2B4852182852283743AF0C2B445
:10079D00D2B5D2B48521828522837455F0C2B4D2EC
:1007AD00B5D2B4852182852283E4F0C2B475171BBE
:1007BD007518009000B11204B5C2B5D2B48521826E
:1007CD0085228374B7F0C2B4D2B5D2B485218285A7
:1007DD0022837407F0C2B4C2B5D2B48521828522BA
:1007ED00837411F0C2B490009612040DC2B5D2B448
:1007FD008521828522837429F0C2B49001F41204FC
:10080D000DA92987060987071EBEFF011F8E198FA7
:10081D001AA92A87060987071EBEFF011F8E1B8F87
:10082D001CE4F517F5189000000205D0AE82AF83D9
:10083D008E048F050CBC00010D8C198D1AAC2BADDF
:10084D002C0CBC00010D8C1B8D1C852B17852C18B9
:10085D008E828F831205D0C2B5D2B48521828522B6
:10086D0083742CF0C2B4AF2ED2B5D2B4852182855B
:10087D002283EFF0C2B4AF2DD2B5D2B485218285DB
:10088D002283EFF0C2B4228582358583367401C38D
:10089D009531FCE49532FD8C378D388531178532D5
:1008AD001890FFFE12133DAA82AB83A831A932E541
:1008BD0031252FF52BE5323530F52C85332D85344B
:1008CD002E853582853683C003C002C001C000125B
:1008DD000839E52FC39531F52BE5309532F52C858B
:1008ED00332D85342E853582853683120839E531D1
:1008FD002535F582E5323536F583852F2B85302C60
:10090D0085332D85342E120839E535C39531F582A1
:10091D00E5369532F583852F2B85302C85332D8546
:10092D00342E120839D000D001D002D003E4F53BAB
:10093D00F53C753901F53AC3E53B98E53C64808992
:10094D00F063F08095F0400122E53820E71618B8E5
:10095D00FF011974022AFAE43BFBEA2537F537EB60
:10096D003538F538C002C003053BE4B53B02053C04
:10097D0074022539F539E4353AF53AE5392537F577
:10098D0037E53A3538F538AC35AD36E53B2CFEE577
:10099D003C3DFF8E3D8F3EAA2FAB30E82AFEE93B52
:1009AD00FF8E3F8F40853F2B85402C85332D853421
:1009BD002E853D82853E83C005C004C003C002C0A4
:1009CD0001C000120839D000D001D002D003D004EC
:1009DD00D005ECC3953BFEED953CFF8E418F4285D6
:1009ED003F2B85402C85332D85342E8541828542C4
:1009FD0083C005C004C003C002C001C00012083985
:100A0D00D000D001D002D003D004D005EAC398FEA7
:100A1D00EB99FF8E2B8F2C85332D85342E853D82C2
:100A2D00853E83C007C006C005C004C003C002C018
:100A3D0001C000120839D000D001D002D003D0047B
:100A4D00D005D006D0078E2B8F2C85332D85342ED7
:100A5D00854182854283C005C004C003C002C00128
:100A6D00C000120839D000D001D002D003D004D07C
:100A7D0005E82CFEE93DFF8E418F42E53B2AFEE560
:100A8D003C3BFF8E2B8F2C85332D85342E8541825B
:100A9D00854283C007C006C005C004C003C002C0A4
:100AAD0001C000120839D000D001D002D003D0040B
:100ABD00D005D006D007ECC398FCED99FD8E2B8F99
:100ACD002C85332D85342E8C828D83C005C004C0BA
:100ADD0003C002C001C000120839D000D001D002FD
:100AED00D003EAC3953BFAEB953CFB8A2B8B2C8507
:100AFD00332D85342E854182854283C003C002C0CB
:100B0D0001C000120839D000D001D002D003D004AA
:100B1D00D0058A2B8B2C85332D85342E8C828D839D
:100B2D00C003C002C001C000120839D000D001D0EE
:100B3D0002D003D003D002020944858245AD457E23
:100B4D0000ED2DFBEE33FCA9298702098707ED2A5D
:100B5D00F546EE3FF547A92A8707098702ED2FF5E0
:100B6D0048EE3AF5497A007D00C3EA9546ED64807A
:100B7D008547F063F08095F050547E007F00C3EE02
:100B8D009548EF64808549F063F08095F050378A81
:100B9D00828D838E2F8F308545317532008543339D
:100BAD00854434C007C006C005C004C003C002128E
:100BBD000894D002D003D004D005D006D007EB2E78
:100BCD00FEEC3FFF80B8EB2AFAEC3DFD809B22AE98
:100BDD0082AF83A9298704098705C3EE9CEF9D5039
:100BED0010A92A8704098705C3E54A9CE54B9D405A
:100BFD000122E54C2EFCE54D3FFD1CBCFF011DA95E
:100C0D00298702098703C3EC9AED9B4010A9298718
:100C1D0004098705ECC39EF54CED9FF54DE54E257A
:100C2D004AFCE54F354BFD1CBCFF011DA92A87026F
:100C3D00098703C3EC9AED9B4012A92A8704098703
:100C4D0005ECC3954AF54EED954BF54FE54C2EFC55
:100C5D00E54D3FFD1CBCFF011D8C198D1AE54E2580
:100C6D004AFCE54F354BFD1CBCFF011D8C1B8D1C3B
:100C7D00854A17854B188E828F831205D0C2B5D247
:100C8D00B4852182852283742CF0C2B4D2B5AF51C4
:100C9D00AD4EAE4FED4E6034AB4CAC4DEB4C6025D4
:100CAD00D2B5D2B4852182852283EFF0C2B4AA5089
:100CBD00D2B5D2B4852182852283EAF0C2B41BBBA2
:100CCD00FF011C80D71DBDFF011E80C822A92887EA
:100CDD0006098707A9288706A92987040987051CFE
:100CED00BCFF011D8C198D1AA92A87040987051CC3
:100CFD00BCFF011D8C1B8D1CE4F517F51890000031
:100D0D00C007C0061205D0D006D007C2B5D2B48533
:100D1D002182852283742CF0C2B4D2B5D2B4852140
:100D2D0082852283EFF0C2B4D2B5D2B485218285FB
:100D3D002283EEF0C2B4D2B47CB07D048C028D035C
:100D4D001CBCFF011DEA4B60467B1085218285226C
:100D5D0083EFF0852182852283EEF0852182852225
:100D6D0083EFF0852182852283EEF0852182852215
:100D7D0083EFF0852182852283EEF0852182852205
:100D8D0083EFF0852182852283EEF0DBBE80AD7D81
:100D9D003F8D041DEC6012852182852283EFF08545
:100DAD002182852283EEF080E8C2B422858252A989
:100DBD00238753098754A9248755098756A927875F
:100DCD0057098758A928875909875AA925875B7418
:100DDD0001B55B0474018001E4FA8A5FE557B559EA
:100DED0008E558B55A03D38001C39200755C0074B1
:100DFD0005B55C05755E00802F855217751800903E
:100E0D000005C00212133DAD82AE83D002ED248EDB
:100E1D00FDEE3414FEE55CFC3395E0FFEC2DF58220
:100E2D00EF3EF583E493F55EC2D5E55B30E704B2A2
:100E3D00D5F404F5F0E55C30E704B2D5F404A43044
:100E4D00D50AF42401C5F0F43400C5F0FEAFF08EE0
:100E5D00048F05755D00E55E20E003020F42EA6038
:100E6D005AC004C005E55CF5603395E0F561AC53FF
:100E7D00AD54E5602CFCE5613DFD8C828D83E55D17
:100E8D00F5603395E0F561AC55AD56E5602CFCE5AC
:100E9D00613DFD8C2B8D2C85572D85582EC007C09F
:100EAD0006C005C004C002120839D002D004D00516
:100EBD00D006D007D005D004021021C002AA53AB32
:100ECD0054EC2AFAED3BFB8A828B83C2D5E55B306D
:100EDD00E704B2D5F404F5F0E55D30E704B2D5F4DE
:100EED0004A430D50AF42401C5F0F43400C5F0F59E
:100EFD006085F061AA55AB56E5602AFAE5613BFBCA
:100F0D008A4A8B4BE55BFA3395E0FB8A4C8B4D8A15
:100F1D004E8B4F855750855851C007C006C005C030
:100F2D0004C002120BDCD002D004D005D006D007CD
:100F3D00D002021021300003021021E55F605AC07B
:100F4D0004C005E55CF5603395E0F561AC53AD5437
:100F5D00E5602CFCE5613DFD8C828D83E55DF560E2
:100F6D003395E0F561AC55AD56E5602CFCE5613D82
:100F7D00FD8C2B8D2C85592D855A2EC007C006C092
:100F8D0005C004C002120839D002D004D005D00625
:100F9D00D007D005D004021021C004C005AB53AD5D
:100FAD0054EE2BFBEF3DFD8B828D83C2D5E55B307F
:100FBD00E704B2D5F404F5F0E55D30E704B2D5F4FD
:100FCD0004A430D50AF42401C5F0F43400C5F0F5BD
:100FDD006085F061AB55AD56E5602BFBE5613DFDE0
:100FED008B4A8D4BE55BFC3395E0FD8C4C8D4D8C28
:100FFD004E8D4F855950855A51C007C006C005C04A
:10100D0004C002120BDCD002D004D005D006D007EC
:10101D00D005D004E55EC313F55E055DC3E55D64E3
:10102D008094885003020E63055CC3E55C64809474
:10103D00865003020DFC22AF82BF0A31A924A824D9
:10104D008605088606A8258604E4C40354F8CCC496
:10105D0003CC6CCC54F8CC6CFBEC2DFDEB3EFEA719
:10106D000509A706E523F8760008760022BF0D01D5
:10107D00228F82120DB9A923A8238606088607A8F8
:10108D002586058D17751800900006C007C006C08F
:10109D000112133DAC82AD83D001D006D007EC2EEA
:1010AD00FEED3FFFA70609A70722AD82AE83AFF085
:1010BD007B007C00EB2DF8EC3EF98F028882898352
:1010CD008AF01213A7FA60208A82C007C006C005F5
:1010DD00C004C003121044D003D004D005D006D0F4
:1010ED00070BBB00CF0C80CC22AF827D007E00BFF2
:1010FD000100405F8F037C0075170A8C188B828C62
:10110D0083C006C005C004C0031213C3A982AA83FD
:10111D00D003D00475170A7518008B828C83C0021A
:10112D00C0011213F9AB82D001D002D005D0068BCD
:10113D00078D178E1890000AC007C002C001121348
:10114D003DAB82AC83D001D002D007E92BFDEA3C48
:10115D00FE809C8D828E83221210F6AE82AF838E1E
:10116D00048F05C3EC9401ED9400404275170A7588
:10117D0018008C828D83C005C00412135AAA82D028
:10118D0004D00575170A7518008C828D83C0021264
:10119D001314AC82AD83D0028C068D0774302AF502
:1011AD0082C007C006121044D006D00780B122AF0E
:1011BD0082E4F562F563740F5FFEEFC4540FFFEE2A
:1011CD0024F640098E0574302DF56280197D007569
:1011DD00170A8D188E828D83C0071213C3AD82D06E
:1011ED000774412DF563EF24F640098F0674302EF8
:1011FD00F56280157E0075170A8E188F828E831208
:10120D0013C3AE8274412EF563856382121044853B
:10121D006282021044E528F876000876F8120CDA9E
:10122D0090001412040DE528F876E0087607120CEC
:10123D00DA90001412040D758200120536E528F8B7
:10124D007600087600120CDA7543007544F8758245
:10125D0014120B4790006412040D120CDA758205FE
:10126D00120522E4F517F5189007FF12050D9019D8
:10127D008975F0801210B7758203120522901992AC
:10128D0075F0801210B790199D75F0801210B790FF
:10129D00009612040D120CDA758201120536E4F572
:1012AD0017F5189000001204F89019A875F0801227
:1012BD0010B790009612040D120CDA758202120509
:1012CD0036E4F517F5189000001204F89019B3756F
:1012DD00F0801210B790009612040D120CDA758280
:1012ED0003120536E4F517F5189000001204F89076
:1012FD00009612040D9019BE75F0801210B7900073
:07130D009612040D020CDA38
:10148E0000000000003E5B4F5B3E3E6B4F6B3E1C10
:10149E003E7C3E1C183C7E3C181C577D571C1C5E27
:1014AE007F5E1C00183C1800FFE7C3E7FF001824FE
:1014BE001800FFE7DBE7FF30483A060E26297929A8
:1014CE0026407F050507407F05253F5A3CE73C5ADD
:1014DE007F3E1C1C08081C1C3E7F14227F22145FBA
:1014EE005F005F5F06097F017F006689956A606015
:1014FE0060606094A2FFA29408047E040810207E0F
:10150E00201008082A1C08081C2A08081E10101093
:10151E00100C1E0C1E0C30383E3830060E3E0E06D9
:10152E00000000000000005F00000007000700142C
:10153E007F147F14242A7F2A1223130864623649EB
:10154E005620500008070300001C224100004122D3
:10155E001C002A1C7F1C2A08083E080800807030D8
:10156E000008080808080000606000201008040247
:10157E003E5149453E00427F40007249494946214D
:10158E0041494D331814127F1027454545393C4AC1
:10159E0049493141211109073649494936464949D8
:1015AE00291E000014000000403400000008142220
:1015BE00411414141414004122140802015909068E
:1015CE003E415D594E7C1211127C7F494949363E8F
:1015DE00414141227F4141413E7F494949417F0975
:1015EE000909013E414151737F0808087F00417F80
:1015FE0041002040413F017F081422417F4040407E
:10160E00407F021C027F7F0408107F3E4141413E15
:10161E007F090909063E4151215E7F091929462697
:10162E004949493203017F01033F4040403F1F209B
:10163E0040201F3F4038403F631408146303047872
:10164E0004036159494D43007F4141410204081092
:10165E0020004141417F04020102044040404040CD
:10166E00000307080020545478407F28444438383B
:10167E0044444428384444287F38545454180008AD
:10168E007E090218A4A49C787F0804047800447D87
:10169E0040002040403D007F1028440000417F4024
:1016AE00007C047804787C08040478384444443878
:1016BE00FC1824241818242418FC7C080404084858
:1016CE005454542404043F44243C4040207C1C20A9
:1016DE0040201C3C4030403C44281028444C909004
:1016EE00907C4464544C440008364100000077005E
:1016FE0000004136080002010204023C2623263C6B
:10170E001EA1A161123A4040207A385454555921F5
:10171E0055557941225454784221555478402054DD
:10172E005579400C1E52721239555555593954542B
:10173E00545939555454580000457C410002457D9A
:10174E00420001457C407D1211127DF0282528F0C3
:10175E007C545545002054547C547C0A097F4932F0
:10176E00494949323A4444443A324A4848303A4167
:10177E0041217A3A42402078009DA0A07D3D424210
:10178E00423D3D4040403D3C24FF2424487E494399
:10179E00662B2FFC2F2BFF0929F620C0887E09030C
:1017AE0020545479410000447D413048484A323833
:1017BE004040227A007A0A0A727D0D19317D26295F
:1017CE00292F28262929292630484D402038080857
:1017DE00080808080808382F10C8ACBA2F1028348B
:1017EE00FA00007B000008142A142222142A14087E
:1017FE00AA005500AAAA55AA55AA000000FF00107B
:10180E001010FF00141414FF001010FF00FF101032
:10181E00F010F0141414FC001414F700FF0000FF75
:10182E0000FF1414F404FC141417101F10101F10D2
:10183E001F1414141F00101010F0000000001F10D1
:10184E001010101F10101010F010000000FF1010DC
:10185E0010101010101010FF10000000FF140000E8
:10186E00FF00FF00001F10170000FC04F4141417F3
:10187E0010171414F404F40000FF00F714141414D9
:10188E00141414F700F7141414171410101F101F4B
:10189E00141414F4141010F010F000001F101F0098
:1018AE0000001F14000000FC140000F010F01010D7
:1018BE00FF10FF141414FF141010101F000000006E
:1018CE00F010FFFFFFFFFFF0F0F0F0F0FFFFFF0062
:1018DE0000000000FFFF0F0F0F0F0F384444384475
:1018EE00FC4A4A4A347E02020606027E027E0263E9
:1018FE00554941633844443C04407E201E20060274
:10190E007E020299A5E7A5991C2A492A1C4C720150
:10191E00724C304A4D4D303048784830BC625A4691
:10192E003D3E494949007E0101017E2A2A2A2A2A82
:10193E0044445F444440514A444040444A5140006C
:10194E0000FF0103E080FF000008086B6B083612F1
:10195E00362436060F090F06000018180000001076
:10196E0010003040FF0101001F01011E00191D175C
:10197E0012003C3C3C3C000000000057656C636F5D
:10198E006D650A004543454E2D3433330A0000522F
:10199E006F746174696F6E203000526F7461746978
:1019AE006F6E203100526F746174696F6E20320059
:0B19BE00526F746174696F6E2033007B
:101314007A10E4FBFCE58225E0F582E58333F5836E
:10132400EB33FBEC33FCEB9517F5F0EC951840062A
:09133400FCABF0438201DADD227A
:06003500E478FFF6D8FD9F
:100013007900E94400601B7A009019C9780175A042
:1000230000E493F2A308B8000205A0D9F4DAF2754C
:02003300A0FF2C
:10133D00E5828517F0A4C582C0F08518F0A4D0F021
:10134D0025F0C5838517F0A42583F58322E5174580
:10135D001860467A01E51725E0F517E518334012B8
:10136D00F518E5829517E583951840030A80E6C3C5
:10137D00E51813F518E51713F517C3E5829517F55D
:10138D00F0E58395184005F58385F082C3E51813C4
:0A139D00F518E51713F517DAE12241
:10003B007800E84400600A790175A000E4F309D860
:10004B00FC7800E84400600C7900900001E4F0A318
:04005B00D8FCD9FAFA
:0D000600758163121431E58260030200036E
:1013A70020F71430F6148883A88220F507E6A8836F
:1013B70075830022E280F7E49322E022C2D5E58319
:1013C70030E70DD2D5E4C39582F582E49583F583A2
:1013D700E51830E70BE4C39517F517E49518F518EA
:1013E70012135A30D50BE4C39582F582E49583F541
:1013F7008322C2D5E58330E70DD2D5E4C39582F5C4
:1014070082E49583F583E51830E70DB2D5E4C395FB
:1014170017F517E49518F51812131430D50BE4C314
:0E1427009582F582E49583F58322758200227A
:00000001FF
